:10000000DBC04CC2F4C0F3C0F2C0F1C0F0C0EFC01E
:10001000EEC0EDC0ECC0EBC0EAC0E9C0E8C0E7C08C
:10002000E6C0E5C0E4C0120368007500730061001B
:100030006B002E0070006C00040309040A033100F9
:1000400030003000320005010905A1010901A100BD
:1000500009300931150026FF00750895028102C09C
:100060000509190129081500250175019508810266
:10007000C01201010100000008100801E5000300A2
:1000800002030105010905A1010901A100093009C7
:1000900031150026FF00750895028102C005091977
:1000A000012904150025017501950481027501954A
:1000B000048103C005010905A1010901A10009305E
:1000C0000931150026FF00750895028102C0050957
:1000D0001901290815002501750195088102C01232
:1000E00001010100000008100801E50003010203FE
:1000F00001120101010000000810089D0A00030020
:1001000002030105010904A1010901A100850109FA
:10011000300931150026FF00750895028102050996
:100120001901290815002501750195088102C0C033
:1001300005010904A1010901A10085020930093165
:10014000150026FF0075089502810205091901298D
:100150000815002501750195088102C0C005010937
:1001600004A1010901A10085030930093115002608
:10017000FF0075089502810205091901290815007B
:100180002501750195088102C0C005010904A1017E
:100190000901A100850409300931150026FF007509
:1001A0000895028102050919012908150025017524
:1001B0000195088102C0C00011241FBECFE5D4E024
:1001C000DEBFCDBF12E0A0E6B0E0E0E1F6E102C0A4
:1001D00005900D92AA32B107D9F722E0AAE2B2E067
:1001E00001C01D92A53AB207E1F757D80FCA08CF50
:1001F000CF93C62F20917A0224FF1CC020917B024E
:1002000038E8232720937B02ECE7F2E09C01D90138
:100210002F5F3F4F9C9191939C2F921B980F191623
:10022000B4F36C2F8CE792E035D1CC5FC0937A02A7
:10023000CF9108952AE520937A02E6CFCF93DF93FA
:1002400080918B02835087FD27C0909187029D3259
:1002500009F58830F9F480918802CCE0D0E0C81B21
:10026000D109C157DD4F83EC80936F028AE58093FB
:10027000610010922A028881807609F460C0CE0164
:1002800075D29F81911104C09E81981708F4892F1F
:100290008093600010928B028091610084FF42C0C5
:1002A000809160008F3F09F43DC0C82F893008F06D
:1002B000C8E0982F9C1B9093600090916F0228E8F3
:1002C000922790936F02882301F180918902909187
:1002D0008A0220912A0226FFAFC0FC012C2F40E7A2
:1002E00052E03491DA013C934F5F5F4F31962150D9
:1002F000C1F79C012F5F3F4F8FEF8C0F820F932F21
:10030000911D90938A02809389026C2F80E792E07E
:10031000C1D084E08C0FC83019F09FEF909360003B
:100320008093610084E190B3957031F48150D9F7E6
:1003300010928C0210928602DF91CF9108952A814B
:1003400010927802998191110AC01092790228E7DF
:1003500032E082E030938A022093890292CF953076
:1003600029F420938C0228E732E0F4CF963009F08C
:100370004CC09B81913019F4CE01CAD144C0923057
:1003800031F4CE01C5D190E090932A027ACF933018
:1003900061F5211109C088E390E090938A0280936F
:1003A000890290E484E0F0CF213049F486E290E0C5
:1003B00090938A028093890290E482E1E5CF223013
:1003C00049F484E890E090938A028093890290E057
:1003D00084E2DACF2330B9F48CE390E090938A0280
:1003E0008093890290E48CE0CFCF913249F48DE381
:1003F00092E090938A028093890290E489E0C4CFCE
:10040000923209F4B9CF90E4BFCF983071F09930AF
:1004100019F420938E02A7CF9A3059F09B3009F03F
:10042000A2CF9BE490937B029ECF2EE832E081E046
:1004300091CF28E732E0FBCFDC012C2F40E752E0E0
:10044000FA013D9130834F5F5F4F2150C9F751CF83
:1004500085B7826085BF8BB780648BBFEAE7F2E027
:100460008BE481838AE580830895A82FB92F80E0EB
:1004700090E041E050EA609530E009C02D9182277C
:100480009795879510F084279527305EC8F36F5FA6
:10049000A8F30895EADF8D939D930895CF93CFB786
:1004A000CF93C395809BE9F7809B09C0809B07C0D1
:1004B000809B05C0809B03C0809B01C0A3C0DF93CD
:1004C000C0918802DD27C157DD4F809B02C0DF91BC
:1004D000EBCF2F930F931F9300B32FEF00FB20F967
:1004E0004F933F9310B34FEF012700FB21F93BE0FF
:1004F00031C04E7F012F10B3216028C0102F4D7FD7
:100500002260000000B329C04B7F2460012F00004F
:1005100010B32BC010B3477F28602AC04F7E00B3B2
:1005200020612CC04F7D10B320622FC04F7B00B3E1
:10053000206432C0422700B349934FEF00001027D8
:1005400010FB20F910B31570C9F1297F91F2012732
:1005500000FB21F900B3237F89F2315058F11027B5
:1005600010FB22F910B3277E79F2012700FB23F953
:100570002F7C81F200B3102710FB24F92F7971F240
:1005800000C010B3012700FB25F92F7359F200C0FA
:1005900000B3102710FB26F9223040F200C010B340
:1005A000012700FB27F9243028F64F77206810B385
:1005B0000000F9CF10E41ABF002719C03B50319555
:1005C000C31BD04010E41ABF0881033CF9F00B3480
:1005D000E9F0209186021981110F1213EDCF4A81A3
:1005E000441F093641F10D3211F0013E29F7009305
:1005F0008D023F914F911F910F912F91DF91CAB7BB
:10060000C6FD4FCFCF91CFBFCF91189520918D02CE
:10061000222379F310918B02112369F534306AF1AA
:1006200030938B0220938702109188023BE0311BAC
:100630003093880222C000918B020130E4F40AE575
:100640004F7049F43091610034FD19C0009361008E
:10065000CFE6D2E018C030917A0234FD10C000938A
:100660007A02CBE7D2E00FC02795A8F45150A9F445
:10067000220F0000F9CF4AE503C042ED01C0432F2D
:10068000C4E1D0E032E011B31560909A11BB02B31F
:1006900020E415E05F93012756E002BB279520F484
:1006A000515021F4220FF9CF012756E000003B5AA8
:1006B00002BBD0F2279528F4515029F4220F0000F4
:1006C000F9CF012756E0279502BB20F4515021F4C1
:1006D000220FF9CF012756E02991332302BB21F6DF
:1006E0000A7F10918C02110FC651D04002BB11F04D
:1006F0001093860210E41ABF016011B31A7F402FD5
:100700004A7F5F9100C000C002BB11BB42BB71CFEA
:10071000FC018081807641F59181963031F593819D
:100720009230D1F0923269F09130F9F48091430225
:100730009091440290938A028093890280914202B0
:100740000895809146029091470290938A02809387
:10075000890280914502089582E690E090938A0292
:100760008093890282E2089580E00895DC018CE2A2
:1007700092E090938A02809389028C9180768032F5
:1007800011F080E0089511968C911197823081F0DC
:100790008A30F1F08130A9F7E0914002F0914102F6
:1007A0000088F189E02D12966C918CE292E0099418
:1007B00012968C919FEF980F983018F78150990BF3
:1007C0008E5C9D4F90938A028093890281E0089508
:1007D0001296EC911297E1110BC0E2E3F2E013964E
:1007E0008C911397819382E0EA33F807C1F7C9CF60
:1007F0008FEF8E0F883028F613968C91F0E0EF5C27
:10080000FD4F8083BECF8091A600882321F01092F7
:10081000A60081E0089580E00895FC01892B09F489
:100820003BC02091490230914A02832F807F803F54
:10083000A9F581E080934802422F50E09FEF20FF0E
:1008400090E821FD90E08FEF22FF80E823FD80E01B
:1008500090838183CA0165E0959587956A95E1F754
:100860008270BA01A3E075956795AA95E1F7647067
:10087000862B221F2227221F822B559547954870D1
:10088000842B828390914802911106C090E1399F98
:1008900090011124822B828383E0089510924802F4
:1008A000CBCFAC9A20E32A95F1F7AC9898E080E0A2
:1008B00028E12A95F1F7AD98880F9B9B816028E18C
:1008C0002A95F1F7AD9A915099F78093490298E0F3
:1008D00028E12A95F1F7AD9886959B9B806828E1E1
:1008E0002A95F1F7AD9A915099F780934A020895AD
:1008F000CF93CFB7F894A49AA59AA398AB9AAD9A40
:10090000AC98CFDFCFBF80E0CF91089586E490E030
:100910009093AC008093AB0087EA90E0089508952F
:1009200080914E02811109C081E020914D02909189
:100930004C02291303C080E0089581E00895FC0172
:1009400020914D0220934C02892B31F1422F50E02F
:100950009FEF20FF90E821FD90E08FEF22FF80E8DD
:1009600023FD80E090838183CA0135E095958795CA
:100970003A95E1F78270BA01A3E075956795AA955B
:10098000E1F76470862B221F2227221F822B5595A8
:1009900047954870842B828383E008958091CF002F
:1009A0008111C29A20E32A95F1F7C29898E080E07D
:1009B00020E32A95F1F728B330914B0231111EC084
:1009C00037EF232328BB880F26B330E040914B023A
:1009D00062E070E0442311F068E070E026233723E2
:1009E000232B09F4816028B338E0411131E0232B37
:1009F00028BB9150E9F680934D0208953EEFE1CF78
:100A0000CF93DF93BA9A87B390914B02911175C03F
:100A100098E0892B87BB84B390914B0291116FC0F2
:100A200090E2892B84BB87B390914B02911169C0EE
:100A30009DEF892387BB88B390914B02911163C0CE
:100A400092E0892B88BB88B390914B0291115DC0D5
:100A500098E0892B88BBC29885B390914B02911185
:100A600056C090E2892B85BB84B390914B029111C3
:100A700050C090E2892B84BB80914B028823C1F047
:100A8000A89A84B390914B02911145C090E2892BB2
:100A900084BBC498BC9A80914B02882349F02FE70D
:100AA00089EA93E0215080409040E1F700C00000C7
:100AB000D1E0D093CF0072DFC0914D021092CF00F1
:100AC0006DDFD093CF0090914B02911102C0C032E4
:100AD00031F1C11104C080914D028F3F01F184B307
:100AE00091111BC09FED892384BB80914B02882309
:100AF00011F0BC98C49A81E013C091E08ACF91E0D4
:100B000090CF97EF96CF98E09CCF91E0A2CF91E065
:100B1000A9CF91E0AFCF91E0BACF9EEFE4CF80E0D4
:100B2000DF91CF910895EBEBF0E083E890E09583BF
:100B3000848381E790E091878087CF01089583B314
:100B400026B34091AD01322F3F70922F9072413009
:100B500069F0932B86958071892B453069F494E078
:100B6000299F900111242074822B0895892F832BB3
:100B70002071822B20E382270895FC01892B49F004
:100B80008091530290915402A091550280839183E9
:100B9000A2838091530290915402A09155028093B8
:100BA000500290935102A093520283E00895EF9275
:100BB000FF920F931F93CF93DF93EC018091AD01D0
:100BC00010E000E0823058F5A498AC9A8D98959A80
:100BD00088EC8A95F1F783B3182F107184FF04C055
:100BE00080914F02882391F081E080934F02A7DF2C
:100BF000111101C08F7D88838FEF89838A83DF91F4
:100C0000CF911F910F91FF90EF900895A49AAC9A05
:100C10008D98959AE8E7EA95F1F791DFECCFA49AE1
:100C2000AC9A8D98959AF8E7FA95F1F7F02E0111A4
:100C300022C085DF8883AC98A49A8D989598E8E7C0
:100C4000EA95F1F7F3E0FF1661F0C8010296F110A2
:100C500002C081E090E07E01E80EF91E70DFF7012E
:100C600080830F5F1F4F04301105C9F6A49AAC9A18
:100C70008D98959AC4CF83E00813DDCF60DF8A8317
:100C8000DACF8091D000882321F01092D00081E04B
:100C9000089543E050E060E572E083E592E0A9D476
:100CA00008951F93CF93DF93C4E6D0E010E047DFB1
:100CB00085FF11C0DF5F88E28A95F1F7C150B9F76F
:100CC000123220F0C1E0D23208F4C0E08C2FDF9164
:100CD000CF911F9108951F5FEECF86E886B986E019
:100CE00087B9089587B9369A08953699FECF84B1A9
:100CF00095B10895F7DFF9CF8F929F92AF92BF928F
:100D0000CF92DF92EF92FF920F931F93CF93DF93D7
:100D1000CDB7DEB72A970FB6F894DEBF0FBECDBFB2
:100D20008091AD01823009F078C08FE088BBE3E5A7
:100D3000CE2EE2E0DE2EF9EEEF2EF0E0FF2E05EEF5
:100D400010E086E08E838E81D5DF70E4972EB12C83
:100D5000A12C9A9491105CC0950150E040E060E0B5
:100D600070E080E490E023D421153105F1E04F07D5
:100D7000510580F5C901F701608171812617370798
:100D800010F431832083F80160817181681779073D
:100D900010F431832083F70180819181281B390B66
:100DA000410951098824922EA32EB42E8F82988651
:100DB000A986BA86F80120813181281B390B50E0C1
:100DC00040E0C501B401F3D32F3F31054105510582
:100DD00029F020F02FEF30E040E050E0F6012193C1
:100DE0006F01F2E0EF0EF11C0E5F1F4F8E81873016
:100DF00061F486B390E0809590959595879595954B
:100E0000879583708093550263C0E7E0EE839BCFA4
:100E10008E8170DFA80EB91E9CCF853009F06BC0A3
:100E200010915602012F0170E1E010FDE0E0F0E0CA
:100E3000ED5AFD4F80E880831092550280DE84FDDC
:100E400005C090915502916090935502807411FFF6
:100E50000AC0811105C080915502826080935502BD
:100E600084E0E82E19C08111FBCF8091550281608A
:100E7000F5CFF8E0FA95F1F7115059F060DE85FFF3
:100E8000F8CF5DDE182FE8E0EA95F1F758DE85FD32
:100E900005C0EA94EE20E1F014E6F0CF88EF8A95E1
:100EA000F1F74DDE85FDF5CF4ADEF82EE8E0EA9554
:100EB000F1F745DE85FDEDCF1295107F8F2D8F70F8
:100EC000812B01118095E02FF0E0ED5AFD4F8083DA
:100ED0002A960FB6F894DEBF0FBECDBFDF91CF913B
:100EE0001F910F91FF90EF90DF90CF90BF90AF9048
:100EF0009F908F900895CE01019659DE9981892F98
:100F000080952A814B8190FD2DC090E081FD9FEF5F
:100F100030E082FF30E883FD3FEF3093530290933F
:100F200054025091AD01382F3071982F9072533088
:100F3000D8F0209524FB882780F931118260911127
:100F4000846025FD8860543009F05CCF942F909523
:100F500042FF806191FD806290FD806493FF52CFDB
:100F6000806850CF90E8D2CF81E0311101C080E09D
:100F7000992309F447CF826045CF1F93CF93DF9326
:100F800000D000D00F92CDB7DEB71FB7F894A59868
:100F9000AD9A87B3807C87BB88B38F6388BBA49AE4
:100FA000AC9A87EB9BE00197F1F700C0000086B395
:100FB000807329F4A59A81E08093AD0124C0BC9A86
:100FC0009FE729EA33E0915020403040E1F700C02C
:100FD000000067DE8823D1F085E08093AD0182E0D8
:100FE0008093560289DE109256028091550280FF4E
:100FF00003C091E09093560281FF05C08091560294
:101000008260809356021FBF80E00BC0CE01019624
:10101000CEDD1092AD0189818F70833059F41FBFEE
:101020008FEF0F900F900F900F900F90DF91CF9157
:101030001F9108958F30C9F48A818F708330A9F48D
:101040008C818F70833021F48D818F70833009F013
:1010500084E08093AD018A8185FD03C084E08093A4
:10106000AD014ADED0CF16B8F6CFA49AAC9A8FE085
:1010700088BB80E387BB17BA30DE86E03BDE86E0C4
:1010800039DE48973CF087E035DE9C0191E028315D
:1010900031050CF490E08FE388BB80E387BB17BA7F
:1010A0008FEB24ED31E0815020403040E1F700C06B
:1010B00000009923C1F282E07FCF84EB90E090930F
:1010C000D6008093D50081ED90E0089582E190E014
:1010D00008959FB7F894B99AC198BD9AC59AA09AF5
:1010E000A89A84B3817C84BB85B38E6385BB9FBF84
:1010F00080E008950F931F93CF93DF93CDB7DEB7B2
:1011000062970FB6F894DEBF0FBECDBFA8988BE2F2
:1011100091E00197F1F700C00000FE01319690E0E8
:10112000AF013FE090FF41C0C59A999BFECF83B3CA
:1011300026B3822F869580712F70822B832781930F
:10114000ABE2B1E01197F1F700C000009F5F923170
:1011500049F7C59AA89A89818F30E1F48A818F3046
:10116000C9F48E010D5F1F4F30E020E086E0F801EA
:1011700091918F019E30E9F09F30E9F492E0D9011E
:10118000AD59BD4F980F891318C02D5F3F4F2C30BC
:10119000310569F762960FB6F894DEBF0FBECDBF7A
:1011A000DF91CF911F910F910895C5989999FECF26
:1011B000BECF93E0E4CF90E0E2CFBA01680F711D9B
:1011C000FB0160816D938F5FDECFCF93DF93EC01E6
:1011D000862F662309F43CC0262F660F330B21505F
:1011E0003109D901AA0FBB1FA20FB31FAD014D5981
:1011F0005D4FA95ABD4F93E0FA0101900D929A9567
:10120000E1F7FA01908130E090FF30E891FD3FEF87
:1012100060E092FF60E893FD6FEFFA012181922F69
:10122000917020FD92E021FD946022FD916023FDEC
:101230009860FA01228120FD906421FD906222FDD8
:10124000906123FD9068888369833A839B8384E05F
:10125000DF91CF9108959091AE01992321F01092E2
:10126000AE0181E00895815023E08202C001112483
:10127000BC01695A7D4F43E050E08D599D4FB9D173
:101280000895EFEAF1E083E091E09583848381EFB4
:1012900090E091878087CF010895CDB7DEB7AA97F8
:1012A0000FB6F894DEBF0FBECDBF7E0123E2E20E83
:1012B000F11C88E0D701E82F1D92EA95E9F7E2E3F7
:1012C000F2E0DF011D928A95E9F717BA8FE388BB38
:1012D000E7EBFBE03197F1F700C0000010924B0202
:1012E00022DCFC0190934102809340020284F3854A
:1012F000E02D0995811113C082E2E3ECF1E0DE01FB
:10130000119601900D928A95E1F782E2FE013196E5
:10131000A4E8B0E001900D928A95E1F737C081E032
:1013200080934B0200DCFC019093410280934002C9
:101330000284F385E02D0995811104C082E2E5EE77
:10134000F1E0DDCFBADEFC019093410280934002D0
:101350000284F385E02D0995882309F4B6C082E262
:10136000E7E0F2E0DE01119601900D928A95E1F737
:1013700082E2FE013196A4E8B0E001900D928A95D8
:10138000E1F77FDF9093410280934002E0914002B9
:10139000F0914102848195819093470280934602A7
:1013A00082818093450280859185009709F499C0D8
:1013B00090934402809343028681809342028091FD
:1013C000450280937B0014BA8FEF85BB88E182BB16
:1013D00085E081BB11BA83BF8FE085BD84EC83BDFE
:1013E00085B78F7885BFE0914002F0914102028479
:1013F000F385E02D09952CD87894CC24C3949924B6
:101400009394AA24A394B12C90E8892E0C2DA8952E
:1014100015D7002341F0E0914002F091410204848D
:10142000F585E02D0995E0914002F0914102028896
:10143000F389E02D309709F0099588B7082F0170DE
:1014400080FF0FC098BEE0914002F09141026081A0
:10145000718130E000E0832F90E0861797070CF44D
:1014600048C008B607FE2AC088BEE0914002F0914D
:10147000410282899389892B69F485B7806885BF89
:10148000889585B78F7785BF8BE291E00197F1F75B
:1014900000C00000E0914002F09141020484F58513
:1014A000E02D099510E0C12ED12CE0914002F09181
:1014B000410280819181C816D906A4F1002309F464
:1014C000A6CFD12CC12C10E059C0E091AD0120E293
:1014D000E29FF0011124E351FF4F80E2A6E8B0E063
:1014E00019CF8FED90E09093440280934302EEDD9C
:1014F00064CFFC01EE5CFD4F4081442341F0F701D5
:10150000E80FF91F2081253020F0255020833F5F10
:10151000A2CF4083A50102C0440F551F8A95E2F770
:10152000042BF5CF1F5F0684F785E02D812F0995E9
:10153000882309F4B8CFC50101C0880FCA94EAF71F
:10154000082BB1CFD394D80102C0B595A7958A9541
:10155000E2F7A0FF13C080917A0284FF0FC00088D9
:10156000F189E02D6D2D8AE392E00995682F8AE3D9
:1015700092E03ED680917A0284FF0CC08D2D90E0DF
:10158000E0914002F091410220813181821793075E
:10159000CCF23CCF53D6A895E0914002F0914102A5
:1015A0000288F389E02D309729F30995E3CFA1E272
:1015B0001A2EAA1BBB1BFD010DC0AA1FBB1FEE1FCD
:1015C000FF1FA217B307E407F50720F0A21BB30B18
:1015D000E40BF50B661F771F881F991F1A9469F794
:1015E00060957095809590959B01AC01BD01CF01F0
:1015F0000895FB01DC0104C08D910190801921F454
:1016000041505040C8F7881B990B0895F894FFCFBC
:10161000FF5A090222000101000032090400000102
:101620000300000009211001000122340007058198
:101630000308000A22032800530029004E00450039
:1016400053002F00410074006100720069005F00C8
:101650005500530042000101002B00000000000073
:10166000007804510403040D04000001003100005F
:1016700000120000000005CE0490049F048F0401B6
:101680000101002B00000000000000BD077C0641A6
:1016900006BD050000020202027F007F00530054D5
:1016A0000044005F003200420054004E005F0055CD
:1016B00000530042002D004A004F005900410074C1
:1016C0000061007200690037006B0038005F005550
:1016D00000530042002D004A004F005900580050AE
:1016E000006100640064006C00650073005F0055D9
:1016F00000530042002D004A004F0059005300657E
:1017000000670061003300420054004E005F005546
:1017100000530042002D004A004F0059005300655D
:1017200000670061003600420054004E005F005523
:1017300000530042002D004A004F00590048004469
:101740000050002D003200300030004A005F00558C
:1017500000530042002D004A004F005900FF0104D1
:1017600000B40000001200000069087A082B09E5A7
:1017700008000022034E00450053002F00420035B0
:1017800000300031005F005500530042002D004A38
:10179000004F00590022034E00450053002F004225
:1017A000003500300033005F005500530042002D2B
:1017B000004A004F00590022035300650067006192
:1017C000004D0075006C00740069007400610070C9
:0A17D000005F0055005300420000C6
:00000001FF
